:10E0000031400003B240805A20013F4002000F938C
:10E0100005242F839F4F4CE30002FB233F40020067
:10E020000F9304241F83CF430202FC23304008E3F4
:10E03000304034E00013B2900A002E010124001396
:10E04000B1C0D0000000FB3F0F120E12D2432100DE
:10E05000E2B302000F24E2C302003E40FF000F4E75
:10E060003F50F1FF0E4F1F93FA37E2B30200F32344
:10E07000824F02023E413F4100130E430E9F052C8A
:10E08000034303431E530E9FFB2B30410B120A1216
:10E090000A4F0B430B9F072C3F40FF0FB0127AE053
:10E0A0002B520B9AF92B3A413B41304192C360010C
:10E0B000B240007D720182437001B2D01200600153
:10E0C00032D0D000B2F0EDFF6001824370013041E8
:10E0D000B240805A2001C2432100C2432900C243FA
:10E0E0002600D2432E00F240FBFF2200F240F8FF50
:10E0F0002A00C2432400C2432C00C2432500C2436D
:10E100002D00F2D040005700E2C302003F40FF0064
:10E110003F50F1FF1F93FC37E2B30200F523F2D02A
:10E1200088FF5800E2D30000B24000016001824342
:10E1300070013041D2434A00B2401000B001B240F9
:10E140001000B2013041E2B228000324B01270E1A5
:10E150003041B01258E130413F43B0127AE0D2D39F
:10E1600021003F43B0127AE0D2C32100F53F304195
:10E170000B120A1209120A430B434943B2D003009F
:10E18000B00192B3B201FD23B2902D01B4010A385F
:10E1900059933024D2D321003F406400B0128CE068
:10E1A000D2C321000E4A0F4B3E800F000F7315346F
:10E1B000E2B22000E3235943D2D321003F43B012FF
:10E1C0007AE03F43B0127AE03F43B0127AE03F4337
:10E1D000B0127AE0D2C32100D13FF2C221003F4306
:10E1E000B0127AE0D2D321003F43B0127AE0D2C31A
:10E1F0002100F53FF2D0030021003F406400B0123F
:10E200008CE0E2C321003F40F401B0128CE0D2C3A5
:10E2100021001A530B63C63F39413A413B4130411B
:10E220000B124B43B2D00300B00192B3B201FD23F5
:10E23000B2900002B4010A345B931D24D2D32100B2
:10E240003F406400B0128CE0D2C32100E2B2200053
:10E25000E9235B43D2D321003F43B0127AE03F432E
:10E26000B0127AE03F43B0127AE03F43B0127AE056
:10E27000D2C32100D73FF2D003002100F2C2210017
:10E280003F406400B0128CE0E2C3210032D0F000C5
:10E29000FD3F3B4130410B124B43B2D00300B00174
:10E2A00092B3B201FD23B2900102B4010A385B932C
:10E2B0001D24D2D321003F406400B0128CE0D2C3B1
:10E2C0002100E2B22000E9235B43D2D321003F4387
:10E2D000B0127AE03F43B0127AE03F43B0127AE0E6
:10E2E0003F43B0127AE0D2C32100D73FF2D00300FF
:10E2F00021003F406400B0128CE0E2C3210032D024
:10E30000F000FD3F3B41304131400003B012D0E00E
:10E31000B01234E13F40D007B0128CE0F2D22100BD
:10E320003F40FF0FB0127AE0E2B328000924E2B2C6
:10E3300028000324B01220E2FF3FB01296E2FC3F17
:0CE34000B01246E1F93F30404AE3FF3FD5
:02E34C000100CE
:10FFE00030E030E030E030E030E030E030E030E091
:10FFF00036E030E030E030E030E030E048E000E093
:040000030000E00019
:00000001FF
